 SwiCEAux

 Timestamp is 54004918 (Fri Aug 29 17:34:16 2014)

 Preferred load address is 10000000

 Start         Length     Name                   Class
 0001:00000000 00003690H .text                   CODE
 0001:00003690 00000060H .text$yc                CODE
 0001:000036f0 00000040H .text$yd                CODE
 0002:00000000 00001288H .rdata                  DATA
 0002:00001288 00000078H .xdata                  DATA
 0002:00001300 00000000H ATL$__a                 DATA
 0002:00001300 00000000H ATL$__z                 DATA
 0002:00001300 00000028H .idata$2                DATA
 0002:00001328 00000014H .idata$3                DATA
 0002:0000133c 000000bcH .idata$4                DATA
 0002:000013f8 000000faH .idata$6                DATA
 0002:00001500 0000017cH .edata                  DATA
 0003:00000000 000000bcH .idata$5                DATA
 0003:000000bc 00000004H .CRT$XCA                DATA
 0003:000000c0 00000004H .CRT$XCAA               DATA
 0003:000000c4 00000004H .CRT$XCL                DATA
 0003:000000c8 00000004H .CRT$XCU                DATA
 0003:000000cc 00000004H .CRT$XCZ                DATA
 0003:000000d0 00000004H .CRT$XIA                DATA
 0003:000000d4 00000004H .CRT$XIZ                DATA
 0003:000000d8 00000004H .CRT$XPA                DATA
 0003:000000dc 00000004H .CRT$XPZ                DATA
 0003:000000e0 00000004H .CRT$XTA                DATA
 0003:000000e4 00000004H .CRT$XTZ                DATA
 0003:000000e8 0000003cH .data                   DATA
 0003:00000128 00000269H .bss                    DATA
 0004:00000000 000002c0H .pdata                  DATA
 0005:00000000 000000a0H .rsrc$01                DATA
 0005:000000a0 000003d0H .rsrc$02                DATA

  Address         Publics by Value              Rva+Base       Lib:Object

 0000:00000000       ___safe_se_handler_count   00000000     <absolute>
 0000:00000000       ___safe_se_handler_table   00000000     <absolute>
 0001:00000008       ?Init@CComCriticalSection@ATL@@QAAJXZ 10001008 f i CEHWIntf.obj
 0001:00000068       ??0CCEHWIntf@@QAA@XZ       10001068 f   CEHWIntf.obj
 0001:0000015c       ?ConnectToBIOS@CCEHWIntf@@QAAJXZ 1000115c f   CEHWIntf.obj
 0001:000003c4       ?DisConnectFromBIOS@CCEHWIntf@@QAAXXZ 100013c4 f   CEHWIntf.obj
 0001:0000041c       ?StartListeningForEvents@CCEHWIntf@@QAAHP6AXPAUSwiNotifyVariant@@@Z@Z 1000141c f   CEHWIntf.obj
 0001:00000428       ?StopListeningForEvents@CCEHWIntf@@QAAXXZ 10001428 f   CEHWIntf.obj
 0001:00000434       ?GetHWAuxVersion@CCEHWIntf@@QAAXPADG@Z 10001434 f   CEHWIntf.obj
 0001:000004bc       ?SetHWPower@CCEHWIntf@@UAAJW4SWIHW_TYPE_Power@@@Z 100014bc f   CEHWIntf.obj
 0001:00000594       ?GetHWAudioPath@CCEHWIntf@@UAAHPAK@Z 10001594 f   CEHWIntf.obj
 0001:00000668       ?HWEnableAudio@CCEHWIntf@@UAAHH@Z 10001668 f   CEHWIntf.obj
 0001:000006e8       ?HWSetVolumnLevel@CCEHWIntf@@UAAHKK@Z 100016e8 f   CEHWIntf.obj
 0001:00000774       ?HWInitiateHostBoot@CCEHWIntf@@UAAHK@Z 10001774 f   CEHWIntf.obj
 0001:000007f4       ?HWSetTetheredMode@CCEHWIntf@@UAAHHPAX@Z 100017f4 f   CEHWIntf.obj
 0001:00000864       ?HWSetDevicePowerState@CCEHWIntf@@UAAJKKK@Z 10001864 f   CEHWIntf.obj
 0001:000008ec       ?GetHWPower@CCEHWIntf@@UAAJPAW4SWIHW_TYPE_Power@@@Z 100018ec f   CEHWIntf.obj
 0001:00000970       ??_ECCEHWIntf@@UAAPAXI@Z   10001970 f i CEHWIntf.obj
 0001:00000970       ??_GCCEHWIntf@@UAAPAXI@Z   10001970 f i CEHWIntf.obj
 0001:000009a0       ??1SWISYNCBLOCK@@QAA@XZ    100019a0 f i HWIntf.obj
 0001:000009ac       ??0CHWIntf@@QAA@XZ         100019ac f   HWIntf.obj
 0001:00000a30       ??1CHWIntf@@UAA@XZ         10001a30 f   HWIntf.obj
 0001:00000ab0       ?NotifyCallback@CHWIntf@@QAAXW4SWIHW_TYPE_Power@@@Z 10001ab0 f   HWIntf.obj
 0001:00000b9c       ?WaitForSingleObjectReset@CHWIntf@@QAAKPAXK@Z 10001b9c f   HWIntf.obj
 0001:00000c18       ?GetInternalPowerState@CHWIntf@@IAA?AW4ePowerInternalState@@XZ 10001c18 f   HWIntf.obj
 0001:00000c48       ?GetModemPowerState@CHWIntf@@QAAJPAW4SWIHW_TYPE_Power@@@Z 10001c48 f   HWIntf.obj
 0001:00000d88       ?SetModemPower@CHWIntf@@QAAJW4SWIHW_TYPE_Power@@@Z 10001d88 f   HWIntf.obj
 0001:00001220       ?BlockingAutoSuspend@CHWIntf@@QAAJHPAX@Z 10002220 f   HWIntf.obj
 0001:00001494       ??_GCriticalSection@@UAAPAXI@Z 10002494 f i HWIntf.obj
 0001:00001494       ??_ECriticalSection@@UAAPAXI@Z 10002494 f i HWIntf.obj
 0001:000014c4       ??_ECHWIntf@@UAAPAXI@Z     100024c4 f i HWIntf.obj
 0001:000014c4       ??_GCHWIntf@@UAAPAXI@Z     100024c4 f i HWIntf.obj
 0001:000014e8       DllMain                    100024e8 f   SwiHWAux.obj
 0001:00001530       SwiHWInitialize            10002530 f   SwiHWAux.obj
 0001:00001594       SwiHWUnInitialize          10002594 f   SwiHWAux.obj
 0001:00001600       SwiHWSetPower              10002600 f   SwiHWAux.obj
 0001:00001698       SwiHWGetPower              10002698 f   SwiHWAux.obj
 0001:000016fc       SwiHWGetOEMIDStrA          100026fc f   SwiHWAux.obj
 0001:00001720       SwiHWRegisterCallback      10002720 f   SwiHWAux.obj
 0001:000017a4       HWEnableAudio              100027a4 f   SwiHWAux.obj
 0001:000017f8       HWGetAudioPath             100027f8 f   SwiHWAux.obj
 0001:00001854       HWInitiateHostBoot         10002854 f   SwiHWAux.obj
 0001:000018a8       HWSetVolumnLevel           100028a8 f   SwiHWAux.obj
 0001:000018f8       HWSetTetheredMode          100028f8 f   SwiHWAux.obj
 0001:00001970       ?PowerUpOperation@@YAXPAX@Z 10002970 f   SwiHWAux.obj
 0001:00001988       HWSetDevicePowerState      10002988 f   SwiHWAux.obj
 0001:00001b38       ?SWAI_GetRegValue@@YAJPAUHKEY__@@PBG1AAK@Z 10002b38 f   sw_utilityG:sw_utilityG.dll
 0001:00001b48       ?LogC@@YAXPBGZZ            10002b48 f   sw_utilityG:sw_utilityG.dll
 0001:00001b58       ?LogStoreFileLine@@YAXPAGH@Z 10002b58 f   sw_utilityG:sw_utilityG.dll
 0001:00001b68       ?SWAI_GetRegValue@@YAJPAUHKEY__@@PBG1PAGPAK@Z 10002b68 f   sw_utilityG:sw_utilityG.dll
 0001:00001b78       ?SetRegValue@@YAJPAUHKEY__@@PBG1K@Z 10002b78 f   sw_utilityG:sw_utilityG.dll
 0001:00001b88       ?GetRegValue@@YAJPAUHKEY__@@PBG1AAK@Z 10002b88 f   sw_utilityG:sw_utilityG.dll
 0001:00001b98       memset                     10002b98 f   coredll:COREDLL.dll
 0001:00001ba8       InitializeCriticalSection  10002ba8 f   coredll:COREDLL.dll
 0001:00001bb8       __C_specific_handler       10002bb8 f   coredll:COREDLL.dll
 0001:00001bc8       DeleteCriticalSection      10002bc8 f   coredll:COREDLL.dll
 0001:00001bd8       Sleep                      10002bd8 f   coredll:COREDLL.dll
 0001:00001be8       GetProcAddressW            10002be8 f   coredll:COREDLL.dll
 0001:00001bf8       LoadLibraryW               10002bf8 f   coredll:COREDLL.dll
 0001:00001c08       wcscpy                     10002c08 f   coredll:COREDLL.dll
 0001:00001c18       FreeLibrary                10002c18 f   coredll:COREDLL.dll
 0001:00001c28       _snprintf                  10002c28 f   coredll:COREDLL.dll
 0001:00001c38       WaitForSingleObject        10002c38 f   coredll:COREDLL.dll
 0001:00001c48       free                       10002c48 f   coredll:COREDLL.dll
 0001:00001c58       ??3@YAXPAX@Z               10002c58 f   coredll:COREDLL.dll
 0001:00001c68       EventModify                10002c68 f   coredll:COREDLL.dll
 0001:00001c78       EnterCriticalSection       10002c78 f   coredll:COREDLL.dll
 0001:00001c88       LeaveCriticalSection       10002c88 f   coredll:COREDLL.dll
 0001:00001c98       CreateEventW               10002c98 f   coredll:COREDLL.dll
 0001:00001ca8       _purecall                  10002ca8 f   coredll:COREDLL.dll
 0001:00001cb8       CloseHandle                10002cb8 f   coredll:COREDLL.dll
 0001:00001cc8       WaitForMultipleObjects     10002cc8 f   coredll:COREDLL.dll
 0001:00001cd8       GetTickCount               10002cd8 f   coredll:COREDLL.dll
 0001:00001ce8       DisableThreadLibraryCalls  10002ce8 f   coredll:COREDLL.dll
 0001:00001cf8       GetModuleFileNameW         10002cf8 f   coredll:COREDLL.dll
 0001:00001d08       ??2@YAPAXI@Z               10002d08 f   coredll:COREDLL.dll
 0001:00001d18       CreateThread               10002d18 f   coredll:COREDLL.dll
 0001:00001d28       __security_check_cookie    10002d28     corelibc:armsecgs.obj
 0001:00001d3c       __gsfailure                10002d3c     corelibc:armsecgs.obj
 0001:00001d80       _onexit                    10002d80 f   corelibc:onexit.obj
 0001:00001e2c       atexit                     10002e2c f   corelibc:onexit.obj
 0001:00001e4c       _DllMainCRTStartup         10002e4c f   corelibc:pegdmain.obj
 0001:00001ee4       __security_init_cookie     10002ee4 f   corelibc:seccinit.obj
 0001:00001f34       _cinit                     10002f34 f   corelibc:crt0dat.obj
 0001:000020a4       _cexit                     100030a4 f   corelibc:crt0dat.obj
 0001:000020c0       AtlRawDllMain              100030c0 f   atls:atlbase.obj
 0001:00002158       ?RemoveAll@?$CSimpleArray@PAUHINSTANCE__@@V?$CSimpleArrayEqualHelper@PAUHINSTANCE__@@@ATL@@@ATL@@QAAXXZ 10003158 f i atls:atlbase.obj
 0001:00002194       ??0_ATL_BASE_MODULE70@ATL@@QAA@XZ 10003194 f i atls:atlbase.obj
 0001:000021d8       ??1CAtlBaseModule@ATL@@QAA@XZ 100031d8 f   atls:atlbase.obj
 0001:00002210       ??0CAtlBaseModule@ATL@@QAA@XZ 10003210 f   atls:atlbase.obj
 0001:000022b4       __FrameUnwindToState       100032b4 f   LIBCMT:frame_ce.obj
 0001:0000262c       ?_DestructExceptionObject@@YAXPAUEHExceptionRecord@@E@Z 1000362c f   LIBCMT:frame_ce.obj
 0001:00002698       ?_OffsetToAddress@@YAPAXHPAKK@Z 10003698 f   LIBCMT:frame_ce.obj
 0001:000026e4       ?FindFrameInfo@@YAPAU_FrameInfo@@PAK@Z 100036e4 f   LIBCMT:frame_ce.obj
 0001:00002724       ?FindCatchFrameInfo@@YAPAU_FrameInfo@@PAK@Z 10003724 f   LIBCMT:frame_ce.obj
 0001:00002764       ?_GetRangeOfTrysToCheck@@YAPBU_s_TryBlockMapEntry@@PBU_s_FuncInfo@@HHPAI1@Z 10003764 f   LIBCMT:frame_ce.obj
 0001:00003170       __InternalCxxFrameHandler  10004170 f   LIBCMT:frame_ce.obj
 0001:000032c8       __CxxFrameHandler3         100042c8 f   LIBCMT:frame_ce.obj
 0001:00003300       __GSHandlerCheckCommon     10004300 f   LIBCMT:gshandler.obj
 0001:00003348       __GSHandlerCheck           10004348 f   LIBCMT:gshandler.obj
 0001:00003378       GetCRTStorage              10004378 f   LIBCMT:corecrt.obj
 0001:00003444       _CallSettingFrame          10004444     LIBCMT:handlers_arm.obj
 0001:00003488       ?FindFrameForUnwind@@YAPAKPAKPBU_s_FuncInfo@@@Z 10004488 f   LIBCMT:mdframe_arm.obj
 0001:000034d0       ?FindCatchFrame@@YAPAKPAKK@Z 100044d0 f   LIBCMT:mdframe_arm.obj
 0001:0000351c       ?AdjustFrameForCatch@@YAPAKPAKPBU_s_FuncInfo@@@Z 1000451c f   LIBCMT:mdframe_arm.obj
 0001:00003554       ?GetCurrentState@@YAHPAKPAU_DISPATCHER_CONTEXT@@PBU_s_FuncInfo@@@Z 10004554 f   LIBCMT:ehstate_arm_mips.obj
 0001:000035b0       __report_gsfailure         100045b0 f   coredll:COREDLL.dll
 0001:000035c0       LocalReAlloc               100045c0 f   coredll:COREDLL.dll
 0001:000035d0       LocalAlloc                 100045d0 f   coredll:COREDLL.dll
 0001:000035e0       LocalSize                  100045e0 f   coredll:COREDLL.dll
 0001:000035f0       __security_gen_cookie      100045f0 f   coredll:COREDLL.dll
 0001:00003600       LocalFree                  10004600 f   coredll:COREDLL.dll
 0001:00003610       GetModuleHandleW           10004610 f   coredll:COREDLL.dll
 0001:00003620       strcmp                     10004620 f   coredll:COREDLL.dll
 0001:00003630       ?terminate@std@@YAXXZ      10004630 f   coredll:COREDLL.dll
 0001:00003640       memmove                    10004640 f   coredll:COREDLL.dll
 0001:00003650       TlsCall                    10004650 f   coredll:COREDLL.dll
 0001:00003660       TlsSetValue                10004660 f   coredll:COREDLL.dll
 0001:00003670       TlsGetValue                10004670 f   coredll:COREDLL.dll
 0001:00003680       InterlockedCompareExchange 10004680 f   coredll:COREDLL.dll
 0002:00000000       ??_C@_1O@JDLOHAN@?$AAD?$AAe?$AAl?$AAe?$AAt?$AAe?$AA?$AA@ 10005000     CEHWIntf.obj
 0002:00000010       ??_C@_1BC@GCKHIPE@?$AAN?$AAo?$AAR?$AAe?$AAm?$AAo?$AAv?$AAe?$AA?$AA@ 10005010     CEHWIntf.obj
 0002:00000024       ??_C@_1BI@JFAIJMHL@?$AAF?$AAo?$AAr?$AAc?$AAe?$AAR?$AAe?$AAm?$AAo?$AAv?$AAe?$AA?$AA@ 10005024     CEHWIntf.obj
 0002:0000003c       ??_C@_17LLMMEOJD@?$AAV?$AAa?$AAl?$AA?$AA@ 1000503c     CEHWIntf.obj
 0002:00000044       ??_C@_13OPKGLAFF@?$AAB?$AA?$AA@ 10005044     CEHWIntf.obj
 0002:00000048       ??_C@_13MKMNOPIJ@?$AAD?$AA?$AA@ 10005048     CEHWIntf.obj
 0002:0000004c       ??_C@_13LHMFKAAD@?$AAM?$AA?$AA@ 1000504c     CEHWIntf.obj
 0002:00000050       ??_C@_13HADIAKP@?$AAS?$AA?$AA@ 10005050     CEHWIntf.obj
 0002:000000a8       ??_C@_1CK@KMBMGEBH@?$AAM?$AAo?$AAd?$AAe?$AAm?$AAP?$AAo?$AAw?$AAe?$AAr?$AAO?$AAf?$AAf?$AAS?$AAm?$AAa?$AAr?$AAt?$AAl?$AAy?$AA?$AA@ 100050a8     CEHWIntf.obj
 0002:000000d4       ??_C@_17PNBAHNJB@?$AAS?$AAe?$AAt?$AA?$AA@ 100050d4     CEHWIntf.obj
 0002:000000dc       ??_7CCEHWIntf@@6B@         100050dc     CEHWIntf.obj
 0002:00000100       ??_C@_17FOBECEA@?$AAG?$AAe?$AAt?$AA?$AA@ 10005100     CEHWIntf.obj
 0002:00000108       ??_C@_1CC@BJGAIDMD@?$AAR?$AAI?$AAL?$AA?2?$AAP?$AAo?$AAw?$AAe?$AAr?$AAC?$AAo?$AAn?$AAt?$AAr?$AAo?$AAl?$AA?$AA@ 10005108     CEHWIntf.obj
 0002:0000012c       ??_C@_1BA@OGGJKLHL@?$AAA?$AAu?$AAx?$AAD?$AAL?$AAL?$AA?$DP?$AA?$AA@ 1000512c     CEHWIntf.obj
 0002:0000013c       ??_C@_1BG@HKBJGIIG@?$AAA?$AAU?$AAX?$AA_?$AAD?$AAe?$AAi?$AAn?$AAi?$AAt?$AA?$AA@ 1000513c     CEHWIntf.obj
 0002:00000154       ??_C@_1BC@EJOOAECN@?$AAA?$AAU?$AAX?$AA_?$AAI?$AAn?$AAi?$AAt?$AA?$AA@ 10005154     CEHWIntf.obj
 0002:00000168       ??_C@_1BO@GNEGJLHD@?$AA?4?$AA?2?$AAC?$AAE?$AAH?$AAW?$AAI?$AAn?$AAt?$AAf?$AA?4?$AAc?$AAp?$AAp?$AA?$AA@ 10005168     CEHWIntf.obj
 0002:00000188       ??_C@_1DA@EOCMJMGL@?$AAO?$AAE?$AAM?$AA?5?$AAA?$AAU?$AAX?$AA?5?$AAv?$AAe?$AAr?$AAs?$AAi?$AAo?$AAn?$AA?5?$AAi?$AAs?$AA?5?$AA0?$AAx?$AA?$CF?$AAx?$AA?$AA@ 10005188     CEHWIntf.obj
 0002:000001b8       ??_C@_1BK@OIOAFAID@?$AAG?$AAe?$AAt?$AAA?$AAu?$AAd?$AAi?$AAo?$AAP?$AAa?$AAt?$AAh?$AA?$AA@ 100051b8     CEHWIntf.obj
 0002:000001d4       ??_C@_1BO@NEGBPBBG@?$AAS?$AAe?$AAt?$AAV?$AAo?$AAl?$AAu?$AAm?$AAn?$AAL?$AAe?$AAv?$AAe?$AAl?$AA?$AA@ 100051d4     CEHWIntf.obj
 0002:000001f4       ??_C@_1CC@JLCPFOJP@?$AAI?$AAn?$AAi?$AAt?$AAi?$AAa?$AAt?$AAe?$AAH?$AAo?$AAs?$AAt?$AAB?$AAo?$AAo?$AAt?$AA?$AA@ 100051f4     CEHWIntf.obj
 0002:00000218       ??_C@_1CA@MBMGLBNN@?$AAS?$AAe?$AAt?$AAT?$AAe?$AAt?$AAh?$AAe?$AAr?$AAe?$AAd?$AAM?$AAo?$AAd?$AAe?$AA?$AA@ 10005218     CEHWIntf.obj
 0002:00000238       ??_C@_1BI@IGHKIMNA@?$AAE?$AAn?$AAa?$AAb?$AAl?$AAe?$AAA?$AAu?$AAd?$AAi?$AAo?$AA?$AA@ 10005238     CEHWIntf.obj
 0002:00000250       ??_C@_1BO@OJIEENIE@?$AAA?$AAU?$AAX?$AA_?$AAG?$AAe?$AAt?$AAV?$AAe?$AAr?$AAs?$AAi?$AAo?$AAn?$AA?$AA@ 10005250     CEHWIntf.obj
 0002:00000270       ??_C@_1O@BMNLCBAA@?$AAG?$AAe?$AAt?$AAM?$AAI?$AAO?$AA?$AA@ 10005270     CEHWIntf.obj
 0002:00000280       ??_C@_1O@GDMFJCHH@?$AAS?$AAe?$AAt?$AAM?$AAI?$AAO?$AA?$AA@ 10005280     CEHWIntf.obj
 0002:00000290       ??_C@_1BG@EGMEOML@?$AAO?$AAE?$AAM?$AAA?$AAU?$AAX?$AA?4?$AAd?$AAl?$AAl?$AA?$AA@ 10005290     CEHWIntf.obj
 0002:000002a8       ??_C@_1BM@FFLEOEGO@?$AAA?$AAu?$AAx?$AAA?$AAP?$AAI?$AAD?$AAl?$AAl?$AAN?$AAa?$AAm?$AAe?$AA?$AA@ 100052a8     CEHWIntf.obj
 0002:000002c4       ??_C@_1DI@PCNPOBB@?$AAm?$AA_?$AAp?$AAG?$AAe?$AAt?$AAA?$AAU?$AAX?$AAV?$AAe?$AAr?$AAs?$AAi?$AAo?$AAn?$AA?5?$AAi?$AAs?$AA?5?$AAi?$AAn?$AAv?$AAa?$AAl?$AAi?$AAd?$AA?$AA@ 100052c4     CEHWIntf.obj
 0002:000002fc       ??_C@_02DPKJAMEF@?$CFd?$AA@ 100052fc     CEHWIntf.obj
 0002:00000300       ??_C@_1EE@OOPNGIMI@?$AAR?$AAe?$AAq?$AAu?$AAe?$AAs?$AAt?$AA?5?$AAi?$AAn?$AAv?$AAa?$AAl?$AAi?$AAd?$AA?5?$AAh?$AAw?$AAP?$AAo?$AAw?$AAe?$AAr?$AAS?$AAt?$AAa?$AAt?$AAe?$AA?5?$AA?$DN?$AA?5?$AA?$CF@ 10005300     CEHWIntf.obj
 0002:00000344       ??_C@_1DK@LMOIFBFK@?$AAF?$AAa?$AAi?$AAl?$AA?5?$AAt?$AAo?$AA?5?$AAS?$AAe?$AAt?$AAM?$AAI?$AAO?$AA?5?$AA?$CI?$AAO?$AAN?$AAO?$AAF?$AAF?$AA?0?$AA?5?$AAH?$AAI?$AAG?$AAH?$AA?$CJ?$AA?$AA@ 10005344     CEHWIntf.obj
 0002:00000380       ??_C@_1DI@GHCBOMHG@?$AAF?$AAa?$AAi?$AAl?$AA?5?$AAt?$AAo?$AA?5?$AAS?$AAe?$AAt?$AAM?$AAI?$AAO?$AA?5?$AA?$CI?$AAO?$AAN?$AAO?$AAF?$AAF?$AA?0?$AA?5?$AAL?$AAO?$AAW?$AA?$CJ?$AA?$AA@ 10005380     CEHWIntf.obj
 0002:000003b8       ??_C@_1GA@MDLJOLJH@?$AAG?$AAe?$AAt?$AAA?$AAu?$AAd?$AAi?$AAo?$AAP?$AAa?$AAt?$AAh?$AA?5?$AAr?$AAe?$AAt?$AAu?$AAr?$AAn?$AAs?$AA?5?$AAi?$AAn?$AAv?$AAa?$AAl?$AAi?$AAd?$AA?5?$AAd?$AAw?$AAR@ 100053b8     CEHWIntf.obj
 0002:00000418       ??_C@_1HE@EGECHHBP@?$AAF?$AAa?$AAi?$AAl?$AA?5?$AAt?$AAo?$AA?5?$AAH?$AAW?$AAE?$AAn?$AAa?$AAb?$AAl?$AAe?$AAA?$AAu?$AAd?$AAi?$AAo?$AA?5?$AAb?$AAE?$AAn?$AAa?$AAb?$AAl?$AAe?$AA?5?$AA?$DN?$AA?5@ 10005418     CEHWIntf.obj
 0002:00000490       ??_C@_1LI@LPCOMACO@?$AAF?$AAa?$AAi?$AAl?$AA?5?$AAt?$AAo?$AA?5?$AAH?$AAW?$AAS?$AAe?$AAt?$AAV?$AAo?$AAl?$AAu?$AAm?$AAn?$AAL?$AAe?$AAv?$AAe?$AAl?$AA?5?$AAd?$AAw?$AAT?$AAX?$AAA?$AAu?$AAd@ 10005490     CEHWIntf.obj
 0002:00000548       ??_C@_1FG@DOLIMPKE@?$AAF?$AAa?$AAi?$AAl?$AA?5?$AAt?$AAo?$AA?5?$AAH?$AAW?$AAI?$AAn?$AAi?$AAt?$AAi?$AAa?$AAt?$AAe?$AAH?$AAo?$AAs?$AAt?$AAB?$AAo?$AAo?$AAt?$AA?5?$AAd?$AAw?$AAB?$AAo?$AAo@ 10005548     CEHWIntf.obj
 0002:000005a0       ??_C@_1EG@HJNNGCMH@?$AAE?$AAR?$AAR?$AAO?$AAR?$AA?3?$AA?5?$AAm?$AA_?$AAp?$AAI?$AAn?$AAi?$AAt?$AAi?$AAa?$AAt?$AAe?$AAH?$AAo?$AAs?$AAt?$AAB?$AAo?$AAo?$AAt?$AA?5?$AAi?$AAs?$AA?5?$AAN?$AAU@ 100055a0     CEHWIntf.obj
 0002:000005e8       ??_C@_1IE@KCNKEENH@?$AAF?$AAa?$AAi?$AAl?$AA?5?$AAt?$AAo?$AA?5?$AAH?$AAW?$AAS?$AAe?$AAt?$AAT?$AAe?$AAt?$AAh?$AAe?$AAr?$AAe?$AAd?$AAM?$AAo?$AAd?$AAe?$AA?5?$AAb?$AAE?$AAn?$AAa?$AAb?$AAl@ 100055e8     CEHWIntf.obj
 0002:00000670       ??_C@_1KA@HKAPDHPN@?$AAC?$AAo?$AAu?$AAl?$AAd?$AA?5?$AAn?$AAo?$AAt?$AA?5?$AAf?$AAi?$AAn?$AAd?$AA?5?$AAH?$AAW?$AA?5?$AAP?$AAo?$AAw?$AAe?$AAr?$AA?5?$AAS?$AAt?$AAa?$AAt?$AAe?$AA?5?$AAv?$AAi@ 10005670     CEHWIntf.obj
 0002:00000710       ??_7CriticalSection@@6B@   10005710     HWIntf.obj
 0002:00000714       ??_7CHWIntf@@6B@           10005714     HWIntf.obj
 0002:00000738       ??_C@_1DK@PFMIPBAF@?$AAa?$AAc?$AAt?$AAi?$AAv?$AAe?$AAl?$AAo?$AAw?$AA_?$AAs?$AAw?$AAi?$AAm?$AAd?$AAm?$AAr?$AAe?$AAs?$AAe?$AAt?$AA_?$AAs?$AAi?$AAg?$AAn?$AAa?$AAl?$AA?$AA@ 10005738     HWIntf.obj
 0002:00000774       ??_C@_1DC@HOGOPNOP@?$AAS?$AAW?$AAI?$AA_?$AAm?$AAo?$AAd?$AAe?$AAm?$AA_?$AAn?$AAe?$AAe?$AAd?$AAs?$AA_?$AAs?$AAh?$AAu?$AAt?$AAd?$AAo?$AAw?$AAn?$AA?$AA@ 10005774     HWIntf.obj
 0002:000007dc       ??_C@_1BM@BMGNNND@?$AA?4?$AA?4?$AA?2?$AAH?$AAW?$AAI?$AAn?$AAt?$AAf?$AA?4?$AAc?$AAp?$AAp?$AA?$AA@ 100057dc     HWIntf.obj
 0002:000007f8       ??_C@_1FO@GGIJJNB@?$AAS?$AAW?$AAI?$AA_?$AAT?$AAY?$AAP?$AAE?$AA_?$AAP?$AAo?$AAw?$AAe?$AAr?$AA?5?$AA?$DN?$AA?5?$AA?$CF?$AAd?$AA?0?$AA?5?$AAa?$AAn?$AAd?$AA?5?$AAS?$AAW?$AAI?$AAH?$AAW?$AA_?$AAT@ 100057f8     HWIntf.obj
 0002:000008a0       ??_C@_1KG@EIJCBGJB@?$AAG?$AAe?$AAt?$AAM?$AAo?$AAd?$AAe?$AAm?$AAP?$AAo?$AAw?$AAe?$AAr?$AAS?$AAt?$AAa?$AAt?$AAe?$AA?5?$AAd?$AAe?$AAt?$AAe?$AAc?$AAt?$AAs?$AA?5?$AAi?$AAn?$AAt?$AAe?$AAr@ 100058a0     HWIntf.obj
 0002:00000998       ??_C@_1FK@KHEGLMPE@?$AAS?$AAe?$AAt?$AAH?$AAW?$AAP?$AAo?$AAw?$AAe?$AAr?$AA?3?$AA?5?$AAi?$AAn?$AAt?$AAl?$AAP?$AAo?$AAw?$AAe?$AAr?$AAS?$AAt?$AAa?$AAt?$AAe?$AA?5?$AAn?$AAo?$AAt?$AA?5?$AAc@ 10005998     HWIntf.obj
 0002:000009f8       ??_C@_1BCI@BICHPAFC@?$AAS?$AAe?$AAt?$AAH?$AAW?$AAP?$AAo?$AAw?$AAe?$AAr?$AA?3?$AA?5?$AAF?$AAA?$AAI?$AAL?$AA?$DP?$AA?5?$AAf?$AAi?$AAn?$AAa?$AAl?$AAH?$AAW?$AAP?$AAo?$AAw?$AAe?$AAr?$AAS?$AAt@ 100059f8     HWIntf.obj
 0002:00000b20       ??_C@_1GG@HDCDHMBC@?$AAN?$AAo?$AAD?$AAR?$AA?$CB?$AA?0?$AA?5?$AAw?$AAa?$AAi?$AAt?$AAR?$AAe?$AAs?$AAu?$AAl?$AAt?$AA?5?$AA?$DN?$AA?5?$AA?$CF?$AAd?$AA?4?$AA?5?$AAO?$AAN?$AA_?$AAO?$AAF?$AAF?$AA?5?$AAl@ 10005b20     HWIntf.obj
 0002:00000b88       ??_C@_1DE@GMPBGNFA@?$AAF?$AAa?$AAi?$AAl?$AAs?$AA?5?$AAt?$AAo?$AA?5?$AAS?$AAe?$AAt?$AAH?$AAW?$AAD?$AAr?$AAv?$AAP?$AAo?$AAw?$AAe?$AAr?$AAO?$AAf?$AAf?$AA?$AA@ 10005b88     HWIntf.obj
 0002:00000bc0       ??_C@_1GE@DDKBPCCK@?$AAN?$AAo?$AAD?$AAR?$AA?$CB?$AA?0?$AA?5?$AAw?$AAa?$AAi?$AAt?$AAR?$AAe?$AAs?$AAu?$AAl?$AAt?$AA?5?$AA?$DN?$AA?5?$AA?$CF?$AAd?$AA?4?$AA?5?$AAT?$AAu?$AAr?$AAn?$AA?5?$AAo?$AAf?$AAf@ 10005bc0     HWIntf.obj
 0002:00000c28       ??_C@_1EO@FFHCCIOD@?$AAN?$AAo?$AAD?$AAA?$AA?$CB?$AA?0?$AA?5?$AAw?$AAa?$AAi?$AAt?$AAR?$AAe?$AAs?$AAu?$AAl?$AAt?$AA?5?$AA?$DN?$AA?5?$AA?$CF?$AAd?$AA?0?$AA?5?$AAT?$AAi?$AAc?$AAk?$AAC?$AAo?$AAu?$AAn@ 10005c28     HWIntf.obj
 0002:00000c78       ??_C@_1DG@EEOHBCMN@?$AAD?$AAe?$AAv?$AAi?$AAc?$AAe?$AA?5?$AAa?$AAr?$AAr?$AAi?$AAv?$AAa?$AAl?$AA?5?$AAd?$AAe?$AAt?$AAe?$AAc?$AAt?$AAe?$AAd?$AA?$CB?$AA?$CB?$AA?$CB?$AA?$AA@ 10005c78     HWIntf.obj
 0002:00000cb0       ??_C@_1IK@FPHBGKFP@?$AAR?$AAI?$AAL?$AA?5?$AAs?$AAt?$AAa?$AAr?$AAt?$AAs?$AA?5?$AAt?$AAh?$AAe?$AA?5?$AA?$CF?$AAd?$AA?5?$AAs?$AAe?$AAc?$AAo?$AAn?$AAd?$AAs?$AA?5?$AAt?$AAi?$AAm?$AAe?$AAo?$AAu@ 10005cb0     HWIntf.obj
 0002:00000d3c       ??_C@_1DC@GMPJONFK@?$AAF?$AAa?$AAi?$AAl?$AAs?$AA?5?$AAt?$AAo?$AA?5?$AAS?$AAe?$AAt?$AAH?$AAW?$AAD?$AAr?$AAv?$AAP?$AAo?$AAw?$AAe?$AAr?$AAO?$AAn?$AA?$AA@ 10005d3c     HWIntf.obj
 0002:00000d70       ??_C@_1CE@EOAGABHK@?$AAF?$AAo?$AAr?$AAc?$AAe?$AA?5?$AAP?$AAo?$AAw?$AAe?$AAr?$AA?5?$AAd?$AAo?$AAw?$AAn?$AA?$CB?$AA?$AA@ 10005d70     HWIntf.obj
 0002:00000d98       ??_C@_1FM@JOOOEFGO@?$AAI?$AAn?$AAt?$AAe?$AAr?$AAn?$AAa?$AAl?$AA?5?$AAs?$AAt?$AAa?$AAt?$AAe?$AA?5?$AAi?$AAs?$AA?5?$AAa?$AAl?$AAr?$AAe?$AAa?$AAd?$AAy?$AA?5?$AAo?$AAn?$AA?4?$AA?5?$AAR?$AAe@ 10005d98     HWIntf.obj
 0002:00000df8       ??_C@_1FO@GADNNJLI@?$AAI?$AAn?$AAt?$AAe?$AAr?$AAn?$AAa?$AAl?$AA?5?$AAs?$AAt?$AAa?$AAt?$AAe?$AA?5?$AAi?$AAs?$AA?5?$AAa?$AAl?$AAr?$AAe?$AAa?$AAd?$AAy?$AA?5?$AAo?$AAf?$AAf?$AA?4?$AA?5?$AAR@ 10005df8     HWIntf.obj
 0002:00000e58       ??_C@_1M@IACDNALF@?$AAh?$AAE?$AAv?$AAt?$AA?$DP?$AA?$AA@ 10005e58     HWIntf.obj
 0002:00000e68       ??_C@_1EI@FPBANDCM@?$AAP?$AAo?$AAw?$AAe?$AAr?$AAM?$AAa?$AAn?$AAa?$AAg?$AAe?$AAr?$AA?1?$AAR?$AAe?$AAl?$AAo?$AAa?$AAd?$AAA?$AAc?$AAt?$AAi?$AAv?$AAi?$AAt?$AAy?$AAT?$AAi?$AAm?$AAe?$AAo@ 10005e68     HWIntf.obj
 0002:00000eb0       ??_C@_1KO@KPNMJCFJ@?$AAB?$AAl?$AAo?$AAc?$AAk?$AAi?$AAn?$AAg?$AAA?$AAu?$AAt?$AAo?$AAS?$AAu?$AAs?$AAp?$AAe?$AAn?$AAd?$AA?5?$AAl?$AAR?$AAe?$AAs?$AAu?$AAl?$AAt?$AA1?$AA?5?$AA?$DN?$AA?5?$AA0@ 10005eb0     HWIntf.obj
 0002:00000f60       ??_C@_1CG@OPCBLDNA@?$AAB?$AAa?$AAt?$AAt?$AAS?$AAu?$AAs?$AAp?$AAe?$AAn?$AAd?$AAT?$AAi?$AAm?$AAe?$AAo?$AAu?$AAt?$AA?$AA@ 10005f60     HWIntf.obj
 0002:00000f88       ??_C@_1CC@LFNKHDIA@?$AAA?$AAC?$AAS?$AAu?$AAs?$AAp?$AAe?$AAn?$AAd?$AAT?$AAi?$AAm?$AAe?$AAo?$AAu?$AAt?$AA?$AA@ 10005f88     HWIntf.obj
 0002:00000fb0       ??_C@_1GA@IEAJLIDI@?$AAS?$AAY?$AAS?$AAT?$AAE?$AAM?$AA?2?$AAC?$AAu?$AAr?$AAr?$AAe?$AAn?$AAt?$AAC?$AAo?$AAn?$AAt?$AAr?$AAo?$AAl?$AAS?$AAe?$AAt?$AA?2?$AAC?$AAo?$AAn?$AAt?$AAr?$AAo?$AAl@ 10005fb0     HWIntf.obj
 0002:00001010       ??_C@_1BK@DADDNBGJ@?$AAB?$AAa?$AAt?$AAt?$AAP?$AAo?$AAw?$AAe?$AAr?$AAO?$AAf?$AAf?$AA?$AA@ 10006010     HWIntf.obj
 0002:0000102c       ??_C@_1BI@JPLMFMBC@?$AAE?$AAx?$AAt?$AAP?$AAo?$AAw?$AAe?$AAr?$AAO?$AAf?$AAf?$AA?$AA@ 1000602c     HWIntf.obj
 0002:00001048       ??_C@_1EO@PFEFPDAL@?$AAS?$AAY?$AAS?$AAT?$AAE?$AAM?$AA?2?$AAC?$AAu?$AAr?$AAr?$AAe?$AAn?$AAt?$AAC?$AAo?$AAn?$AAt?$AAr?$AAo?$AAl?$AAS?$AAe?$AAt?$AA?2?$AAC?$AAo?$AAn?$AAt?$AAr?$AAo?$AAl@ 10006048     HWIntf.obj
 0002:00001098       ??_C@_1FA@KNFIBHMI@?$AAO?$AAn?$AA?5?$AAD?$AA?$CF?$AAd?$AA?0?$AA?5?$AAt?$AAr?$AAy?$AA?5?$AAt?$AAo?$AA?5?$AAs?$AAy?$AAn?$AAc?$AA?5?$AAu?$AAp?$AA?5?$AAt?$AAh?$AAe?$AA?5?$AAm?$AAo?$AAd?$AAe?$AAm@ 10006098     SwiHWAux.obj
 0002:000010e8       ??_C@_1GM@HMGGHPNB@?$AAO?$AAE?$AAM?$AA?$CB?$AA?$CB?$AA?$CB?$AA?5?$AAD?$AAe?$AAt?$AAe?$AAc?$AAt?$AA?5?$AAF?$AAo?$AAr?$AAc?$AAe?$AAd?$AA?5?$AAP?$AAo?$AAw?$AAe?$AAr?$AA?5?$AAU?$AAp?$AA?5?$AAr?$AAe@ 100060e8     SwiHWAux.obj
 0002:00001158       ??_C@_1HA@OEGLCNO@?$AAO?$AAE?$AAM?$AA?$CB?$AA?$CB?$AA?$CB?$AA?5?$AAD?$AAe?$AAt?$AAe?$AAc?$AAt?$AA?5?$AAF?$AAo?$AAr?$AAc?$AAe?$AAd?$AA?5?$AAP?$AAo?$AAw?$AAe?$AAr?$AA?5?$AAD?$AAo?$AAw?$AAn?$AA?5@ 10006158     SwiHWAux.obj
 0002:000011c8       ??_C@_1CA@MDOGLIKH@?$AA?4?$AA?4?$AA?2?$AAS?$AAw?$AAi?$AAH?$AAW?$AAA?$AAu?$AAx?$AA?4?$AAc?$AAp?$AAp?$AA?$AA@ 100061c8     SwiHWAux.obj
 0002:000011e8       ??_C@_1GO@FMHHKKAJ@?$AAO?$AAE?$AAM?$AA?$CB?$AA?$CB?$AA?$CB?$AA?5?$AAD?$AAe?$AAt?$AAe?$AAc?$AAt?$AA?5?$AAC?$AAr?$AAi?$AAt?$AAi?$AAc?$AAa?$AAl?$AA?5?$AAP?$AAo?$AAw?$AAe?$AAr?$AA?5?$AAC?$AAo?$AAn@ 100061e8     SwiHWAux.obj
 0002:00001258       GUID_ATLVer30              10006258     atls:atlbase.obj
 0002:00001268       GUID_ATLVer70              10006268     atls:atlbase.obj
 0002:00001278       IID_IPersistStream         10006278     uuid:objidl_i_guid12.obj
 0002:00001300       __IMPORT_DESCRIPTOR_sw_utilityG 10006300     sw_utilityG:sw_utilityG.dll
 0002:00001314       __IMPORT_DESCRIPTOR_COREDLL 10006314     coredll:COREDLL.dll
 0002:00001328       __NULL_IMPORT_DESCRIPTOR   10006328     sw_utilityG:sw_utilityG.dll
 0003:00000000       __imp_CloseHandle          10007000     coredll:COREDLL.dll
 0003:00000004       __imp_memmove              10007004     coredll:COREDLL.dll
 0003:00000008       __imp_?terminate@std@@YAXXZ 10007008     coredll:COREDLL.dll
 0003:0000000c       __imp_strcmp               1000700c     coredll:COREDLL.dll
 0003:00000010       __imp_InterlockedCompareExchange 10007010     coredll:COREDLL.dll
 0003:00000014       __imp_TlsGetValue          10007014     coredll:COREDLL.dll
 0003:00000018       __imp_TlsSetValue          10007018     coredll:COREDLL.dll
 0003:0000001c       __imp_memset               1000701c     coredll:COREDLL.dll
 0003:00000020       __imp_InitializeCriticalSection 10007020     coredll:COREDLL.dll
 0003:00000024       __imp___C_specific_handler 10007024     coredll:COREDLL.dll
 0003:00000028       __imp_DeleteCriticalSection 10007028     coredll:COREDLL.dll
 0003:0000002c       __imp_Sleep                1000702c     coredll:COREDLL.dll
 0003:00000030       __imp_GetProcAddressW      10007030     coredll:COREDLL.dll
 0003:00000034       __imp_LoadLibraryW         10007034     coredll:COREDLL.dll
 0003:00000038       __imp_wcscpy               10007038     coredll:COREDLL.dll
 0003:0000003c       __imp_FreeLibrary          1000703c     coredll:COREDLL.dll
 0003:00000040       __imp__snprintf            10007040     coredll:COREDLL.dll
 0003:00000044       __imp_WaitForSingleObject  10007044     coredll:COREDLL.dll
 0003:00000048       __imp_free                 10007048     coredll:COREDLL.dll
 0003:0000004c       __imp_??3@YAXPAX@Z         1000704c     coredll:COREDLL.dll
 0003:00000050       __imp_EventModify          10007050     coredll:COREDLL.dll
 0003:00000054       __imp_EnterCriticalSection 10007054     coredll:COREDLL.dll
 0003:00000058       __imp_LeaveCriticalSection 10007058     coredll:COREDLL.dll
 0003:0000005c       __imp_CreateEventW         1000705c     coredll:COREDLL.dll
 0003:00000060       __imp__purecall            10007060     coredll:COREDLL.dll
 0003:00000064       __imp_WaitForMultipleObjects 10007064     coredll:COREDLL.dll
 0003:00000068       __imp_GetTickCount         10007068     coredll:COREDLL.dll
 0003:0000006c       __imp_DisableThreadLibraryCalls 1000706c     coredll:COREDLL.dll
 0003:00000070       __imp_GetModuleFileNameW   10007070     coredll:COREDLL.dll
 0003:00000074       __imp_??2@YAPAXI@Z         10007074     coredll:COREDLL.dll
 0003:00000078       __imp_CreateThread         10007078     coredll:COREDLL.dll
 0003:0000007c       __imp___report_gsfailure   1000707c     coredll:COREDLL.dll
 0003:00000080       __imp_LocalReAlloc         10007080     coredll:COREDLL.dll
 0003:00000084       __imp_LocalAlloc           10007084     coredll:COREDLL.dll
 0003:00000088       __imp_LocalSize            10007088     coredll:COREDLL.dll
 0003:0000008c       __imp___security_gen_cookie 1000708c     coredll:COREDLL.dll
 0003:00000090       __imp_LocalFree            10007090     coredll:COREDLL.dll
 0003:00000094       __imp_GetModuleHandleW     10007094     coredll:COREDLL.dll
 0003:00000098       __imp_TlsCall              10007098     coredll:COREDLL.dll
 0003:0000009c       \177COREDLL_NULL_THUNK_DATA 1000709c     coredll:COREDLL.dll
 0003:000000a0       __imp_?GetRegValue@@YAJPAUHKEY__@@PBG1AAK@Z 100070a0     sw_utilityG:sw_utilityG.dll
 0003:000000a4       __imp_?SetRegValue@@YAJPAUHKEY__@@PBG1K@Z 100070a4     sw_utilityG:sw_utilityG.dll
 0003:000000a8       __imp_?SWAI_GetRegValue@@YAJPAUHKEY__@@PBG1PAGPAK@Z 100070a8     sw_utilityG:sw_utilityG.dll
 0003:000000ac       __imp_?LogStoreFileLine@@YAXPAGH@Z 100070ac     sw_utilityG:sw_utilityG.dll
 0003:000000b0       __imp_?LogC@@YAXPBGZZ      100070b0     sw_utilityG:sw_utilityG.dll
 0003:000000b4       __imp_?SWAI_GetRegValue@@YAJPAUHKEY__@@PBG1AAK@Z 100070b4     sw_utilityG:sw_utilityG.dll
 0003:000000b8       \177sw_utilityG_NULL_THUNK_DATA 100070b8     sw_utilityG:sw_utilityG.dll
 0003:000000bc       __xc_a                     100070bc     corelibc:crt0init.obj
 0003:000000cc       __xc_z                     100070cc     corelibc:crt0init.obj
 0003:000000d0       __xi_a                     100070d0     corelibc:crt0init.obj
 0003:000000d4       __xi_z                     100070d4     corelibc:crt0init.obj
 0003:000000d8       __xp_a                     100070d8     corelibc:crt0init.obj
 0003:000000dc       __xp_z                     100070dc     corelibc:crt0init.obj
 0003:000000e0       __xt_a                     100070e0     corelibc:crt0init.obj
 0003:000000e4       __xt_z                     100070e4     corelibc:crt0init.obj
 0003:000000e8       ?HW2SWNotificationPowerMode@@3PAHA 100070e8     HWIntf.obj
 0003:000000fc       ?theSWIHWCR@@3VCriticalSection@@A 100070fc     SwiHWAux.obj
 0003:00000114       __security_cookie_complement 10007114     corelibc:seccook.obj
 0003:00000118       __security_cookie          10007118     corelibc:seccook.obj
 0003:0000011c       _pRawDllMain               1000711c     atls:atlbase.obj
 0003:00000128       ?m_bInitFailed@CAtlBaseModule@ATL@@2_NA 10007128     CEHWIntf.obj
 0003:0000012c       ?thePwrCtrlObj@@3PAVCCEHWIntf@@A 1000712c     CEHWIntf.obj
 0003:00000130       ?g_ModuleName@@3PAGA       10007130     SwiHWAux.obj
 0003:0000033c       ?theHWIntf@@3PAVCCEHWIntf@@A 1000733c     SwiHWAux.obj
 0003:00000340       ?g_hinstThisDll@@3PAXA     10007340     SwiHWAux.obj
 0003:00000344       ?g_IsCriticalPower@@3HA    10007344     SwiHWAux.obj
 0003:00000348       ?gCallBackP@@3P6AXPAUSwiNotifyVariant@@@ZA 10007348     SwiHWAux.obj
 0003:0000034c       ?_pAtlRawDllMain@@3P6AHPAXK0@ZA 1000734c     atls:atlbase.obj
 0003:00000350       ?_AtlModuleInstance@ATL@@3PAUHINSTANCE__@@A 10007350     atls:atlbase.obj
 0003:00000354       ?_AtlBaseModule@ATL@@3VCAtlBaseModule@1@A 10007354     atls:atlbase.obj
 0003:00000388       __onexitend                10007388     <common>
 0003:0000038c       __onexitbegin              1000738c     <common>
 0003:00000390       _exitflag                  10007390     <common>

 entry point at        0001:00001e4c

 Static symbols

 0001:00000124       __unwind$58920             10001124 f   CEHWIntf.obj
 0001:00000b70       __unwind$40450             10001b70 f   HWIntf.obj
 0001:00000d68       __unwind$40577             10001d68 f   HWIntf.obj
 0001:000011d4       __unwind$40704             100021d4 f   HWIntf.obj
 0001:00001fa0       doexit                     10002fa0 f   corelibc:crt0dat.obj
 0001:0000249c       ?CanThisExceptionObjectBeDestructed@@YAEPAUEHExceptionRecord@@E@Z 1000349c f   LIBCMT:frame_ce.obj
 0001:000027e8       ?CallCatchBlock@@YAPAXPAUEHExceptionRecord@@PAKPAU_CONTEXT@@PBU_s_FuncInfo@@PAXHK@Z 100037e8 f   LIBCMT:frame_ce.obj
 0001:00002b80       ?BuildCatchObject@@YAXPAUEHExceptionRecord@@PAKPBU_s_HandlerType@@PBU_s_CatchableType@@@Z 10003b80 f   LIBCMT:frame_ce.obj
 0001:00002d54       ?FindHandler@@YAEPAUEHExceptionRecord@@PAKPAU_CONTEXT@@PAU_DISPATCHER_CONTEXT@@PBU_s_FuncInfo@@H@Z 10003d54 f   LIBCMT:frame_ce.obj
 0001:00003690       ??__EtheSWIHWCR@@YAXXZ     10004690 f   SwiHWAux.obj
 0001:000036b4       ??__E_AtlBaseModule@ATL@@YAXXZ 100046b4 f   atls:atlbase.obj
 0001:000036f0       ??__FtheSWIHWCR@@YAXXZ     100046f0 f   SwiHWAux.obj
 0001:0000370c       ??__F_AtlBaseModule@ATL@@YAXXZ 1000470c f   atls:atlbase.obj
